:020000040000FA
:060000005BEF13F012009B
:060800005BEF13F0120093
:06082A0001002027000080
:08083000000200002700000097
:0808380058EC09F0FB0EDBCFC8
:10084000F3FFDB06F35000090AE0A6EC09F0FA0E0C
:1008500011EC0AF0F3E1151CF1E1010E01D0000EDC
:1008600087EF09F058EC09F03B0EE12402E3E16860
:10087000E652E16E010EDB6A020EDB6AF90EDBCF97
:10088000F6FFFA0EDBCFF7FFFB0EDBCFF8FF080019
:10089000F550DF6EDF5002E1ABEF08F0250EDF5CB4
:1008A00002E09EEF08F0030EDB6A040EDB6A050E21
:1008B000DB6A060EDB6A070EDB6AC0EC08F02D0E61
:1008C000DF5C0CE02B0EDF5C09E0200EDF5C06E055
:1008D000230EDF5C03E0300EDF5C1AE1DF50300AEC
:1008E00014E0130A0FE0030A0AE00B0A05E0060A07
:1008F000E4E1030EDB80E1D7030EDB82DED7030EDB
:10090000DB84DBD7030EDB86D8D7030EDB88D5D795
:100910002A0EDF5C1BE1BCEC08F00AEC09F010E0E9
:10092000030EDB8006680768130EDBCF0BF0140E96
:10093000DBCF0CF086EC11F0040E04C0DBFF03D01B
:10094000130EF3EC08F0C0EC08F00BD0090EDB6AD4
:1009500061EC09F003E0D5EC09F0FAD7090EF3ECED
:1009600008F0030EDBB0DB982E0EDF5C1BE1C0EC61
:1009700008F02A0EDF5C0BE1BCEC08F00AEC09F091
:1009800003E1130E45EC09F0C0EC08F00BD0090EA2
:10099000DB6A61EC09F003E0D5EC09F0FAD7090E47
:1009A00045EC09F0680EDF5C07E1C0EC08F0680E6A
:1009B000DF5C1DE1030E18D0740EDF5C17E07A0EC9
:1009C000DF5C14E0480EDF5C06E0540EDF5C03E001
:1009D0005A0EDF5C02E1020E07D06C0EDF5C03E012
:1009E0006A0EDF5C04E1010E98EC09F0C9DBDF5010
:1009F0006E0A01E17FD31E0A01E192D1200A01E1D2
:100A00008FD13F0A01E149D11A0A01E146D10D0A0D
:100A100001E143D1200A01E140D13A0A01E13DD18F
:100A2000200A01E13AD1260A01E135D10D0A01E19E
:100A300032D11A0A01E1D9D0200A4AE0300A1FE077
:100A4000460A0EE0250A01E083D3D950F90FE96E7A
:100A5000FF0EDA20EA6E010EEE5E000EEE5AEE5A3E
:100A6000A6EC09F0250EE66E95DB03E1151C01E10D
:100A700069D3A2EC09F001E26BD3DB2A69D3080E3B
:100A8000DB6A040EDB50010806E2040EDB046AECAC
:100A900009F0DB508BDB080EDB5009E0030EDB5066
:100AA000010B05E172DB01E04DD3080EDB6A64DB6C
:100AB000EFCFDFFF1AEC0AF003E1151C01E142D38E
:100AC000A2EC09F001E3DB2A60DB01E141D33AD378
:100AD000070EDB5002080FE1E6EC09F0030EADEC67
:100AE00009F00E0EEECFDBFF0F0EEECFDBFF100E88
:100AF000EECFDBFF20D0F70EDBCF17F0F80EDBCF09
:100B000018F0020E175E000E185AF70E17C0DBFF22
:100B1000F80E18C0DBFF17C0E9FF18C0EAFF9DEC14
:100B200009F0166A0E0E14C0DBFF0F0E15C0DBFFB6
:100B3000100E16C0DBFF0E0EDBCFE6FF0F0EDBCF75
:100B4000E6FF100EDBCFE6FFE0EC12F0E552E552D7
:100B5000E552130E05C0DBFF140E06C0DBFF060EC8
:100B6000DB5005E0130EE1EC09F001E26ADB05EC75
:100B70000AF002E2130E37DBC8EC09F006E0040EBF
:100B8000E1EC09F002E2050E2EDB030EDBB005D02E
:100B9000FCDA01E0D7D2080EDB6A090EDB6A0E0E22
:100BA000DBCFF6FF0F0EDBCFF7FF100EDBCFF8FF2A
:100BB0000800F550DF6EDF5014E00BEC0AF011E294
:100BC0001AEC0AF003E1151C01E1BCD2BBDB01E326
:100BD000DB2A090EDB2AD9500E0FE96E000ECBDBA3
:100BE000E7D7D3DA01E1B4D2ADD2C6DA110EEECF37
:100BF000DBFF120EEDCFDBFF110EDBCFE6FF120E97
:100C0000DBCFE6FFD2EC12F0E552E552130EF3CF44
:100C1000DBFF140EF4CFDBFF060EDB5004E0130EF7
:100C2000D0DB01E20EDB05EC0AF002E2130EDBDAA8
:100C3000AFDB05E0040EC5DB02E2050ED4DA030EDD
:100C4000DBB005D0A2DA01E07DD2080EDB6A090E26
:100C5000DB6A110EDBCFE9FF120EDBCFEAFFEFCF2D
:100C6000DFFFDF5014E0D7DB12E2E4DB03E1151C09
:100C700001E168D267DB01E3DB2A090EDB2A110EF2
:100C8000DB2ADBCFE9FF120EE8E3DB2AE6D77DDAC9
:100C900001E15ED257D2030EDB8E070EDB0410E1BA
:100CA00095DB040E5ADB0A0EEECFDBFF0B0EEECF08
:100CB000DBFF0C0EEECFDBFF0D0EEECFDBFF6CD0BB
:100CC000070EDB5003082CE1030EDBAE0DD0B2DAC9
:100CD000020E76DAEFCF14F0156A166A176A14AEB0
:100CE00039D01568166835D0F70EDBCF15F0F80E41
:100CF000DBCF16F0020E155E000E165AF70E15C069
:100D0000DBFFF80E16C0DBFF15C0E9FF16C0EAFFD7
:100D1000EFCF14F00A0E14C0DBFF0B0EDB6A38D0E5
:100D2000070EDB50020809E1030EDBAE04D059DBED
:100D300016AE10D00ED055DB0DD0030EDBAE12D0A8
:100D400079DA020E3DDAF9DA166A176A15AE02D0C0
:100D500016681768E2DA0C0E16C0DBFF0D0E17C01E
:100D6000DBFF1AD0F70EDBCF16F0F80EDBCF17F053
:100D7000020E165E000E175AF70E16C0DBFFF80EB5
:100D800017C0DBFF16C0E9FF17C0EAFFD6DAC5DAE5
:100D90000C0EDB6A0D0EDB6A060EDB5005E1010E60
:100DA000F36E050EF3CFDBFF150EDB6A160EDB6A62
:100DB000D950370F146E000EDA20156E390E14C09C
:100DC000DBFF3A0E15C0DBFF380EDB6A080EDB6A6C
:100DD0000A0EAEDADF50780A12E0200A10E0280A84
:100DE0000CE0200A0AE03F0A06E00D0A02E0200AB1
:100DF00008E1020E05D0080E03D0080EDF26100E03
:100E000097DA030EDBBE02D0DB92DB94DB50800B63
:100E100024E08ADAD890030EEB50000A08E6000EB0
:100E2000EE5C000EEE58000EEE58000EEE5815E285
:100E300013DA09680A680B680C689AEC12F00A0E5B
:100E400000C0DBFF0B0E01C0DBFF0C0E02C0DBFF9E
:100E50000D0E03C0DBFF2D0E08D0030EDBA202D067
:100E60002B0E03D0DBA408D0200EF36E170EF3CFA9
:100E7000DBFF150EDB2A02D0170EDB6A050EDB50F6
:100E800003E1B7D901E189D0040E146E270E156E67
:100E9000000E166E070EDBCF17F0186A196A1A6A71
:100EA00017C009F018C00AF019C00BF01AC00CF0F6
:100EB000D3D905EC13F014500024F36E1550012023
:100EC000F46E16500220F86EF4CFF7FFF3CFF6FF62
:100ED0000800090EF5CFDBFF580EDF5C0FE1610E55
:100EE000F36E090E7BD90AE3200E146E090EDBCFD8
:100EF000E7FF1450E75E090EE7CFDBFF070EDBCFFD
:100F000014F0156A166A176A0FDA14C009F015C0D2
:100F10000AF016C00BF017C00CF0EECF04F0EECFC5
:100F200005F0EECF06F0EFCF07F005EC13F007C0A9
:100F3000EDFF06C0EDFF05C0EDFF04C0EFFF390E69
:100F4000DBCFE9FFDB063A0EDBCFEAFF01E2DB068F
:100F5000090EDBCFEFFF150EDB2A4BD995E1030E0F
:100F6000DBA61DD06F0EDF5C06E1C1D918E3150EBC
:100F7000DB285BDA14D0780EDF5C09E0580EDF5C0A
:100F800006E0620EDF5C03E0420EDF5C08E1020E69
:100F9000F36E160EF3CFDBFF02D0150EDB6A030EE5
:100FA000DB50100B0EE0040EDBCF14F0050EDB500F
:100FB000D880145406E2060EDB5003E1040EDB5029
:100FC00034DA95D90AE2050EDBCFE7FF150EDB50C8
:100FD000E75E050EE7CFDBFF02D0050EDB6A040EED
:100FE000DBCF14F0160E45D9D880145414E2160E37
:100FF000DBCFE6FF150EDBCFE6FF040EDBCFE6FF0F
:10100000050EDB50E552E75CE552D880E754E55227
:10101000D880E7545FD9030EDB50010B0BE1080EBB
:10102000DB5008E0B2D801E08DD0080EDB50BED80E
:10103000080EDB6A170EDB5007E088D9170EF1D9CE
:1010400003E1151C01E17ED0160EDB5016E07ED9BF
:10105000300EE66E9FD802E1151C74E077D9DFCF21
:10106000E6FF58EC12F0E552E552E552F4CF15F0E8
:101070000001F31C02E1151C65E0050EDBCF14F046
:10108000160EDB50D880145409E2050EDBCFE7FFC3
:10109000160EDB50E75E050EE7CFDBFF300EE66E87
:1010A000050ECBD94FE1390EDB2ADBCFE9FF3A0E33
:1010B00001E3DB2ADBCFEAFF090EEFCFDBFFDB50DA
:1010C0000EE044D9090EADD902E1151C3BE0390E02
:1010D000DB2ADBCFE9FF3A0EEDE3DB2AEBD755D86D
:1010E00031E1160EDBCFE6FF080EC3D8E552E72448
:1010F0005DD82ED0070EDB50030A1CE0010A14E075
:10110000030A07E07BD9DBCFEEFF020EDBCFEDFF5A
:101110001FD0F5D8196A17AE02D0186819682CD8F4
:10112000BCD819C0EEFF14D0EAD817BE186824D86E
:10113000B4D80ED063D9DBCFEFFF0AD07BD905E15D
:10114000151C03E1F368F46810D0FCD801E3DB2A36
:1011500079D947EF04F0010EDBCF14F0020EDBCF9C
:1011600015F014C0F3FF15C0F4FF3B0EE15C02E282
:10117000E16AE552E16ECBD029D9020EADEF09F05C
:1011800061D90800F550DF6E1200200EE66E080EE1
:101190001DEF0AF058EC12F0E552E552E552F3CF9C
:1011A00014F0F4CF15F00001F31C1200146E156A50
:1011B000D950010F4DD91450EE261550ED221200D2
:1011C000185E000E195AF70E18C0DBFFF80E19C092
:1011D000DBFF18C0E9FF19C0EAFF1200DBCFF4FF04
:1011E000F350F45C1200DB50E76E040EE7CFDBFF38
:1011F00012000A0EDBCF14F00B0EDBCF15F00C0E35
:10120000DBCF16F00D0EDBCF17F0145015101610B3
:1012100017101200130EEECFDBFF140EEDCFDBFF25
:10122000130EDBCF14F0140EDBCF15F00001800E8F
:1012300015141200F70EDBCF18F0F80EDBCF19F003
:101240001200050EDB50E66ED950130F01D9E5529E
:10125000E750EE6EED6A12000A0EDBCF04F00B0EC3
:10126000DBCF05F00C0EDBCF06F00D0EDBCF07F069
:101270001200DBCFE6FF150EDBCFE6FF050EDB50DD
:10128000E552E724E552E7241200DB50CED8010EE8
:10129000F36E060EF3CFDBFF1200EE50EFCFEAFF46
:1012A000E96E16C0EEFF17C0EEFF18C0EEFF120089
:1012B000D9CFE6FFDACFE6FFE1CFD9FFE2CFDAFF01
:1012C0001200DFCFE6FFE66A29EC13F0E552E552A3
:1012D000F3501200E76E080EE7CFDBFF1200EECFEF
:1012E00014F0EECF15F0EFCF16F0176A1200050ECE
:1012F000DBCF14F0150EDB50D88014541200010E11
:10130000DBCF16F0020EDBCF17F0186A1200E552A1
:10131000E5CFDAFFE7CFD9FF12000A0E14C0DBFFDA
:101320000B0E15C0DBFF1200D9500A0F28EF0AF090
:10133000F36E070EF3CFDBFF1200EECF14F0EFCF0A
:1013400015F01200010EDB2A020E1200FC0EDBCF9C
:10135000E6FFFD0EDBCFE6FF1200145E000E155A0D
:10136000F70E14C0DBFFF80E15C0DBFF14C0E9FF59
:1013700015C0EAFF1200DA20EA6EEF2AEECFF6FF80
:10138000000EEF22EECFF7FFEF22EECFF8FF1200B4
:10139000040EDBCFE6FF130EDB50E552E75C9ADF6D
:1013A000DB5004DF060EDB501200090EDB500A0D85
:1013B000F350DF24D00FE76E090EE7CFDBFFC0EF5D
:1013C00008F0DB50F36E050EEEEF08F0F70EDBCF02
:1013D00014F0F80EDBCF15F01200DFCFE6FFCAEFF6
:1013E00008F028DF030EECDE6FEF09F01CEC04F0D0
:1013F000E552E552E552E55200091200BDDEEE501D
:10140000EFCFEAFFE96E010E1200130EDB50F36E10
:10141000040EEEEF08F0040EDB50F36E090EEEEF53
:1014200008F0DBCFE6FFCAEF08F0E76E050EE7CF66
:10143000DBFF12008BDFEDEF09F0DBCFE6FF86DF8D
:10144000F6EF09F0D950F90FE96EFF0EBBEF09F086
:0A145000E96E000EDA20EA6E1200C9
:06145A00D9CFE6FFE1CF4F
:10146000D9FF040EE126DE6ADE6ADE6ADD6ADD523D
:10147000DD52FD0EDBCF14F0FE0EDBCF15F0166A49
:10148000176A15AE02D016681768D9CFE9FFDACF10
:10149000EAFF030EEB501718E8AE02D0173408D05D
:1014A0001450EE5C1550EE581650EE581750EE588A
:1014B0000FE20C0EE66E3BEC13F0E552D9CFE9FFDC
:1014C000DACFEAFFEE2A000EEE22EE22EE22D1D78C
:1014D000040EE15C02E2E16AE552E16EE552E7CF1B
:1014E000D9FF12000F0EC16E070EB46E936A300E54
:1014F000926E0F0E946EF19E1200D9CFE6FFE1CFEF
:10150000D9FF020EE1268250020B01E0010E080D08
:10151000F3CF16F08250010B040DF3CF15F080507D
:10152000200B01E0010EE824146E8050100B01E046
:10153000010E142415241624DE6EDD6ADECF14F0AD
:10154000DDCF15F014C0F3FF15C0F4FF020EE15C0F
:1015500003E200D0E16AE552E16EE552E7CFD9FF40
:1015600012008092010EE66EE66A77DFE552E552E0
:101570008084010EE66EE66A70DFE552E5528094E3
:10158000010EE66EE66A69DFE552E55212008082DE
:10159000010EE66EE66A61DFE552E5528084010ED7
:1015A000E66EE66A5ADFE552E5528094010EE66E79
:1015B000E66A53DFE552E5521200380E816ED1DF44
:1015C000320EE66EE66A49DFE552E552010E816EA3
:1015D000C8DF320EE66EE66A40DFE552E5520D0ED8
:1015E000816EBFDF320EE66EE66A37DFE552E55206
:1015F000060E816EB6DF320EE66EE66A2EDFE5522B
:10160000E5521200010E816EACDF0A0EE66EE66A4C
:1016100024DFE552E5521200D9CFE6FFE1CFD9FF32
:10162000020E816E9EDF0A0EE66EE66A16DFE55256
:10163000E552FD0EDBCFE6FFFE0EDB50280DF3502A
:10164000E552E724E76EFE0EE7CFDBFFFD0EDB6A17
:10165000FE0EDB50F36EFD0EDBCFF4FFF350F45CB7
:101660000CE2140E816E7DDF010EE66EE66AF5DE99
:10167000E552E552FD0EDB2AEBD7E552E7CFD9FF65
:101680001200D9CFE6FFE1CFD9FFFE0EDB50816E0D
:101690007EDF010EE66EE66AE0DEE552E552E552D7
:1016A000E7CFD9FF1200D9CFE6FFE1CFD9FFFD0E7A
:1016B000DBCFE9FFFE0EDBCFEAFFEF500EE0FD0EC1
:1016C000DBCFE9FFDB2AFE0EDBCFEAFF01E3DB2AFB
:1016D000EF50E66ED6DFE552EAD7E552E7CFD9FF05
:1016E00012000001646B300E926EF00E936EEF0EDE
:1016F000606F60C081FF040E616F6151000821E2DC
:101700006051FE0BE842606F60C081FF050EE66E1F
:10171000E66AA3DEE552E5528150100B09E08150E4
:10172000200B06E08150400B03E08150800B01E16B
:101730000AD80001640502E1655104D06105616FBA
:10174000DCD7CFD71200F00E936E81CF63F000018B
:101750006315626F0F0E6015606F60516211606FEC
:1017600081CF63F0F00E6315626FF00E625D01E0F1
:10177000F7D7936A06D866C065F00001010E646F62
:1017800012000001676B100E675D14E26751EA6A90
:10179000000FE96E020EEA22EF50605D08E167512A
:1017A000EA6A100FE96E020EEA22EFCF66F06729AF
:1017B000676FE9D766C081FF640EE66EE66A4DDEAC
:1017C000E552E55212000001686B070E685D1DE2EC
:1017D00088DF0001696F6851EA6A6A0FE96E000EDE
:1017E000EA2269C0EFFF6851EA6A6A0FE96E000EEB
:1017F000EA22EF50460802E108D004D069C0E6FFB3
:1018000040DFE5520001682BE0D76851EA6A6A0FB1
:10181000E96E000EEA22EF6A12000001686B070E03
:10182000685D16E26851EA6A6A0FE96E000EEA2204
:10183000EF50E66E26DFE55200016829EA6A6A0F7A
:10184000E96E000EEA22EF5001E102D0682BE7D7E3
:101850001200D9CFE6FFE1CFD9FF0E0EE126DE6AF6
:10186000DD6AB6D8CC0EE66EE66AC3D8E552E5521C
:10187000440EE66EE66ABDD8E552E552D9CFE9FFDF
:10188000DACFEAFFEE50ED1006E11ED9F3CFDEFF0E
:10189000F4CFDDFFF3D79CD8CC0EE66EE66AA9D86C
:1018A000E552E552BE0EE66EE66AA3D8E552E55271
:1018B0000BD9020EF3CFDBFF030EF4CFDBFF04D90D
:1018C000040EF3CFDBFF050EF4CFDBFF040EDBCFFE
:1018D00018F0050EDBCF19F018C019F0186A020EC7
:1018E000DB501824146E030EDB501920156E166A97
:1018F000176A15AE02D016681768060E14C0DBFF13
:10190000070E15C0DBFF080E16C0DBFF090E17C05F
:10191000DBFF060EDBCF18F0070EDBCF19F0080E49
:10192000DBCF1AF0090EDBCF1BF018C004F019C092
:1019300005F01AC006F01BC007F061EC0FF005C0FF
:1019400014F006C015F007C016F008C017F00A6AB8
:101950000B6A800E0C6E410E0D6E14C005F015C0A2
:1019600006F016C007F017C008F011EC10F00A0ED0
:1019700005C0DBFF0B0E06C0DBFF0C0E07C0DBFF54
:101980000D0E08C0DBFFC80EE66EE66A66DDE552A6
:10199000E5520A0EDBCF14F00B0EDBCF15F00C0E68
:1019A000DBCF16F00D0EDBCF17F014C004F015C01E
:1019B00005F016C006F017C007F00E0EE15C03E25A
:1019C00000D0E16AE552E16EE552E7CFD9FF12009F
:1019D000926A8096010EE66EE66A3FDDE552E552B8
:1019E000080E926E010EE66EE66A37DDE552E552AC
:1019F0001200D9CFE6FFE1CFD9FF040EE126020E97
:101A0000DB6A030EDB6A020EDBCF14F0030EDBCFC2
:101A100015F0D890155004E6080E145C000E155809
:101A200049E2926A8096020EE66E77EC13F0E55278
:101A3000010EE76EFD0EDBCF14F0FE0EDBCF15F0CE
:101A4000E7501416156A14C0DEFF15C0DDFFD9CFAC
:101A5000E9FFDACFEAFF010EEE1801E1ED5001E1F6
:101A60008086D9CFE9FFDACFEAFFEE50ED1001E131
:101A700080963C0EE66E77EC13F0E552080E926EFF
:101A8000020EE66E77EC13F0E552FD0EDBCF14F09C
:101A9000FE0EDBCF15F0D89015321432FD0E14C0B7
:101AA000DBFFFE0E15C0DBFF020EDB2A030E01E397
:101AB000DB2AA9D7040EE15C02E2E16AE552E16E9D
:101AC000E552E7CFD9FF1200D9CFE6FFE1CFD9FF2A
:101AD000040EE126DE6ADD6ADECF14F0DDCF15F0FC
:101AE000D890155004E6080E145C000E15584BE211
:101AF000926A8096020EE66E77EC13F0E552080EBD
:101B0000926EE66E77EC13F0E552020EDBCF14F026
:101B1000030EDBCF15F0D89015321432020E14C02C
:101B2000DBFF030E15C0DBFF80A610D0800EE76E32
:101B3000020EDBCF14F0030EDBCF15F0E7501412CA
:101B4000020E14C0DBFF030E15C0DBFF80B611D000
:101B50007F0EE76E020EDBCF14F0030EDBCF15F025
:101B6000E7501416156A020E14C0DBFF030E15C0F1
:101B7000DBFF780EE66E77EC13F0E552DF2A010EFC
:101B800001E3DB2AA9D7020EDBCF14F0030EDBCF73
:101B900015F014C0F3FF15C0F4FF040EE15C03E27E
:101BA00000D0E16AE552E16EE552E7CFD9FF1200BD
:101BB00099DC03DD27DD200EE66E020EE66E73DD96
:101BC000E552E55246DE04C073F005C074F006C06D
:101BD00075F007C076F00A6A0B6A100E0C6E410EA3
:101BE0000D6E73C005F074C006F075C007F076C0C6
:101BF00008F064EC10F005C018F006C019F007C03A
:101C00001AF008C01BF00A6A0B6AA00E0C6E400E98
:101C10000D6E18C005F019C006F01AC007F01BC001
:101C200008F011EC10F005C014F006C015F007C064
:101C300016F008C017F00A6A0B6A0C6A420E0D6EA5
:101C400014C005F015C006F016C007F017C008F064
:101C50007BEC0FF005C077F006C078F007C079F094
:101C600008C07AF073C005F074C006F075C007F0C4
:101C700076C008F0D1EC10F006C07BF007C07CF015
:101C80007BC006F07CC007F04CEC0FF005C018F0EC
:101C900006C019F007C01AF008C01BF018C00AF0FF
:101CA00019C00BF01AC00CF01BC00DF073C005F08A
:101CB00074C006F075C007F076C008F07AEC0FF03B
:101CC00005C014F006C015F007C016F008C017F0E4
:101CD0000A6A0B6A200E0C6E410E0D6E14C005F0E0
:101CE00015C006F016C007F017C008F064EC10F03D
:101CF000D1EC10F006C07DF007C07EF07DC0E6FF9D
:101D00007EC0E6FF7BC0E6FF7CC0E6FF150E146ECA
:101D1000270E156E166A14C0E6FF15C0E6FF16C042
:101D2000E6FF7F0EE66E000EE66EB3EC11F0176E66
:101D3000090EE15E1750E66A010EE66E6DDCE552B3
:101D4000E5527F0EE66E000EE66EADDCE552E55222
:101D5000200EE66E96DCE552D60EE66E92DCE5527B
:101D6000430EE66E8EDCE552D00EE66E070EE66E92
:101D70002DEC0AF0E552E55277C005F078C006F088
:101D800079C007F07AC008F0D1EC10F006C07BF003
:101D900007C07CF07BC006F07CC007F04CEC0FF075
:101DA00005C018F006C019F007C01AF008C01BF0F3
:101DB00018C00AF019C00BF01AC00CF01BC00DF0CF
:101DC00077C005F078C006F079C007F07AC008F057
:101DD0007AEC0FF005C014F006C015F007C016F03D
:101DE00008C017F00A6A0B6A200E0C6E410E0D6EC9
:101DF00014C005F015C006F016C007F017C008F0B3
:101E000064EC10F0D1EC10F006C07DF007C07EF05D
:101E10007DC0E6FF7EC0E6FF7BC0E6FF7CC0E6FF3C
:101E2000150E146E270E156E166A14C0E6FF15C047
:101E3000E6FF16C0E6FF7F0EE66E000EE66EB3EC20
:101E400011F0176E090EE15E1750E66A010EE66E9C
:101E50000CEC0BF0E552E5527F0EE66E000EE66EDE
:101E600022DCE552E552200EE66E0BDCE552D60E82
:101E7000E66E07DCE552460EE66E41EC0BF0E552ED
:101E8000D00EE66E070EE66E2DEC0AF0E552E55236
:041E900099D61200CD
:0C1E94000F9E08D00F9E07AE05D0066C14
:101EA000071EE86A07220F8E07C001F006C000F087
:101EB000136A126A8E0E026E036A1CEF11F00F9EF7
:101EC0000CD00F9E07AE09D0046C051E061E071E1F
:101ED000E86A0522062207220F8E07C001F006C01D
:101EE00000F005C013F004C012F09E0E026E036AEB
:101EF0001CEF11F00D7E0F6A58EC11F070EC11F030
:101F00000FB600EF11F00FA20AD00FAA03D00FBE38
:101F100000EF11F00FA40CEF11F009EF11F00FAA70
:101F200005D00FAC0CEF11F009EF11F00FA00AD0A3
:101F30000FA808D00FBE04D00FA402D015EF11F0E7
:101F400019EF11F0126A036A0D50085C116E10E36C
:101F500005C013F006C000F007C001F008C010F083
:101F60000AC005F00BC006F00CC007F00F3A09D00C
:101F70000AC013F00BC000F00CC001F00DC010F04F
:101F8000116C0F9E0FBC0F8E10C002F00FB048EF07
:101F900011F01A0E116048EF11F0026A086A0FA4DE
:101FA00008D0056C061E071E081EE86A06220722D6
:101FB00008220FAC08D0136C001E011E021EE86A36
:101FC000002201220222046A115207E0083407327B
:101FD000063205320432112EF9D705501326065069
:101FE0000022075001220850022204C012F00F9E66
:101FF00002AE0BD0126C131E001E011E021EE86AF8
:1020000013220022012202220F8E02A006D0D880C5
:102010000132003213321232102A10C002F01CEFCB
:1020200011F00F6A58EC11F070EC11F00FB600EFE0
:1020300011F00FA205D00FBA00EF11F007EF11F069
:102040000FBA13EF11F00FA005D00FB800EF11F089
:1020500013EF11F00FB807EF11F0036A7F0E082499
:10206000026EE86A03220D50025EE86A035A1A0EF5
:10207000106E086A126A136A006A016A0A50055EE5
:102080000B50065A0C50075A000E085A09E70A501E
:1020900005260B5006220C500722000E082201D004
:1020A000128AD8900536063607360836D89012368A
:1020B000133600360136102EE1D7075006100510F2
:1020C000D8A4128A1CEF11F00F6A58EC11F070ECD2
:1020D00011F00FB600EF11F00FA205D00FB800EF0E
:1020E00011F007EF11F00FAA05D00FB000EF11F0BB
:1020F00007EF11F00FB002D00FA802D013EF11F0CC
:10210000036A0D500824026EE86A03227E0E025E06
:10211000E86A035A126A136A006A016A0C500702DD
:10212000F4CF01F0F3CF00F00B500702F350132669
:10213000F4500022000E01220C500602F350132628
:10214000F4500022000E01220A500702F35012261A
:10215000F4501322000E002201220B500602F3500D
:102160001226F4501322000E002201220C50050208
:10217000F3501226F4501322000E002201220A50BE
:102180000602F4501226000E1322002201220B50E8
:102190000502F4501226000E1322002201221CEF29
:1021A00011F00F6A58EC11F00FB6DBEF10F00FA230
:1021B0000ED00FB405D07F0E076EFF0E066E1FD037
:1021C000800E076E066A1BD0076A066A18D00FB029
:1021D000FBD78F0E0860EDD77E0E0864F5D78E0E04
:1021E000085C05E0D89007320632082AF8D70FA419
:1021F00006D0066C071EE86A072207AEE5D7120074
:102200007F0E086EFF0E076E066E056E12007F0EC3
:102210000FBEFF0E086E02D07F0E086E800E076E96
:10222000066A056AF3D70FAE04D0800E086E076AFF
:10223000F7D7086A076AF4D701500010131012107C
:10224000F8E003BEF0D701BE0CD002500310EBE063
:10225000D89012361336003601360206D8A003068F
:10226000F2D70350D4E10228D2E012AE11D07F0E93
:10227000121402E113A00CD0132AE86A00220122F2
:1022800007E3D880013200321332022A0228BFE06D
:102290000250C9E013C005F000C006F00134076E1B
:1022A0000230086E0732089E0FBE088E06EF11F04E
:1022B0000736083602E30F840F7E06E10F80086AB6
:1022C000076A066A056A1200082803E0D880073208
:1022D0001200D890073202E10F8212000F8612001E
:1022E0000C360D3602E30F8C0F7E06E10F880D6A67
:1022F0000C6A0B6A0A6A12000D2803E0D8800C32BF
:102300001200D8900C32EAE10F8A120007C013F0D5
:1023100006C012F006500B02F4CF05F0F3CF04F024
:1023200007500C02F4CF07F0F3CF06F00B02F35086
:102330000526F4500622E86A072212500C02F350D8
:102340000526F4500622E86A07220CAEACEF11F025
:102350001250065E1350075A13AE000C0B50065E67
:062360000C50075A000CAE
:0A236600D9CFE6FFDACFE6FFE1CFA2
:10237000D9FFE2CFDAFFE652E652E652E652D950F2
:10238000F90F146EFF0EDA20156E020E14C0DBFF7B
:10239000030E15C0DBFF020EDBCFE6FF030EDBCF23
:1023A000E6FFF90EDBCFE6FFFA0EDBCFE6FFFB0E12
:1023B000DBCFE6FFD950FC0FE66EFF0EDA20E66EAB
:1023C00032EC04F0146E070EE15C02E2E16AE552C1
:1023D000E16E1450F3CFDEFFF4CFDDFFFC0EDBCF58
:1023E000E9FFFD0EDBCFEAFFEF6ADECF14F0DDCFB1
:1023F00015F014C0F3FF15C0F4FF040EE15C02E217
:10240000E16AE552E16EE552E5CFDAFFE7CFD9FFA9
:022410001200B8
:0E2412002A0EF66E080EF76E000EF86E02012E
:102420000900F5502C6F0900F5502D6F03E12C6762
:1024300001D03DD00900F550276F0900F550286FF5
:102440000900F550296F09000900F550E96E0900EF
:10245000F550EA6E090009000900F5502A6F0900DD
:10246000F5502B6F09000900F6CF2EF2F7CF2FF2AF
:10247000F8CF30F227C2F6FF28C2F7FF29C2F8FFD3
:1024800002012A5302E12B5307E00900F550EE6EDA
:102490002A07F8E22B07F9D72EC2F6FF2FC2F7FF63
:1024A00030C2F8FF02012C07000E2D5BBFD71200CF
:1024B000D9CFE6FFDACFE6FFE1CFD9FFE2CFDAFFEF
:1024C000FB0EDBCF14F0FC0EDBCF15F00001800E0D
:1024D00015141AE1FB0EDBCFE9FFFC0EDBCFEAFFA0
:1024E000EECFF3FFEDCFF4FFEE2A000EEF22F3CF95
:1024F000E9FFF4CFEAFFFD0EDBCFEFFFEF50156AE7
:10250000F36E15C0F4FF10D0FB0EDB50FE0806E1A1
:10251000FD0EDBCFE6FF69EC13F005D0FD0EDBCF3F
:10252000E6FF8EEC13F0E552E552E5CFDAFFE7CF98
:04253000D9FF1200BD
:0C25340004500902F3CF00F0F4CF01F0D6
:102540000A02F3500126000EF420026E04500B0222
:10255000F3500226000EF420036E04500C02F350D8
:10256000032605500902F3500126F4500222000E02
:10257000032205500A02F3500226F45003220550AC
:102580000B02F350032606500902F3500226F450C2
:10259000032206500A02F350032607500902F350A3
:0425A00003261200FC
:0C25A400FE0EE3CFE9FFFF0EE3CFEAFFDD
:1025B000F36AF46AEE5203E0F34AF42AFBD71200FE
:1025C000FF0EE3CFF8FFE552FF0EE3CFF7FFE55232
:1025D000FF0EE3CFF6FFE552E66AE66AE66A090017
:1025E000F55209E0FD0EE32A05E1FE0EE32A02E1C1
:1025F000FF0EE32AF4D7FD0EE3CF05F0FE0EE3CF86
:0A26000006F0FF0EE3CF07F0120012
:06260A00036A026A016A86
:10261000006A200EE76ED890043605360636073677
:1026200000360136023603360950005C0A50015864
:102630000B5002580C50035809E30950005E0A5031
:10264000015A0B50025A0C50035A042AE72EE4D7C1
:02265000120076
:0E265200F36AF46AFF0EE124E96EFF0EE22047
:10266000EA6EED6607D02F0EEF6404D03A0EEF60ED
:0626700001D0F32A120064
:0A267600FF0EE3501C6E480E01D069
:102680004C0EE76EE72EFED7E76AE72EFED71C2E2C
:06269000F7D70000120064
:0A269600000EF36E00EE00F0080ED7
:1026A00001D81200EA6002D0EE6AFCD7F350E9606C
:0626B0001200EE6AFCD7E7
:0A26B60012EE40F022EE40F0F86A48
:1026C0000F9C09EC12F08FEC13F0D8EC0DF0FBD757
:0226D0001200F6
:0E26D200FF0EE350ACBA04D0AF6AAB8EAC8AF8
:0E26E000949CACA2FED7AD6EF36EF46A1200AD
:0226EE00FF0EDD
:1026F000E350E84E1200000000D000D000D0E82ED9
:04270000FAD71200F2
:0C270400303132333435363738396162F9
:05271000636465660032
:072715002533642E2564004A
:02271C001200A9
:02271E001200A7
:10272000EEEDEBE7DEDDDBD7BEBDBBB77E7D7B77B5
:1027300030313233343536373839414243444546F7
:0727400054454D50453D00DA
:00000001FF
